:100000000C94EE050C9416060C9416060C94160629
:100010000C94AA230C9416060C9416060C9416063F
:100020000C9416060C9416060C94261B0C94621A5B
:100030000C94AF220C9416060C9416060C9416061B
:100040000C9416060C9416060C9416060C941606C0
:100050000C9416060C946E220C9416060C9416063C
:100060000C9416060C9416060C9416060C941606A0
:100070000C9416060C9416060C9416060C94160690
:100080000C9416060C9416060C9416060C94160680
:100090000C9416060C9416060C9416060C94160670
:1000A0000C9416060C9416060C941606270C270CB6
:1000B000590C590CCB0C800E800E800EE70CD20D23
:1000C000E30DE30DDC16DC16D416D016D816E816B0
:1000D000E216CA167A18A118441AA118441AED1883
:1000E0001019441A051A141A00F6010002F601004C
:1000F00001F60100642700000DF601002DF6010055
:100100000AF6010012F6010018F6010095F401004C
:1001100029F601004CF4010014F601000FF601006D
:100120007B26000009F601004DF401004EF40100A9
:100130004FF601000CF60100B6F3010033F60100A2
:100140004CF6010022F601000EF6010048F601000F
:1001500049F601004AF60100A9F4010040F401004B
:100160000C27000094F4010034F6010005F60100AC
:10017000AFF4010015F601001CF601001EF60100A7
:100180000BF601004FF4010031F6010008F6010002
:1001900007F601004BF401000026000014F30100F3
:1001A00080F401009103000092030000930300001B
:1001B00094030000950300009603000097030000DD
:1001C00098030000990300009A0300009B030000BD
:1001D0009C0300009D0300009E0300009F0300009D
:1001E000A0030000A1030000A3030000A40300007B
:1001F000A5030000A6030000A7030000A803000059
:10020000A9030000B1030000B2030000B303000023
:10021000B4030000B5030000B6030000B7030000FC
:10022000B8030000B9030000BA030000BB030000DC
:10023000BC030000BD030000BE030000BF030000BC
:10024000C0030000C1030000C3030000C40300009A
:10025000C5030000C6030000C7030000C803000078
:10026000C9030000C20300006422000065220000F0
:1002700060220000B1000000362F231C4241403FA5
:10028000373E141B101112133D3C3B3A39383534BC
:10029000333231302D2C2B2526272021221D1E1FE5
:1002A00018191A1516172E243C393431211E191627
:1002B000000000000000000000000000000000003E
:1002C000000000000000000000000000000000002E
:1002D000000000007E0F00D4FFFFFFC70000007881
:1002E00000000000000000002A2B28000000000091
:1002F00000000000000000000000002900000000D5
:100300002C1E3420212224342627252E362D373842
:10031000271E1F202122232425263333362E37384B
:100320001F0405060708090A0B0C0D0E0F10111209
:10033000131415161718191A1B1C1D2F3130232DD5
:10034000350405060708090A0B0C0D0E0F101112D3
:10035000131415161718191A1B1C1D2F3130354C84
:1003600005010980A101850319012AB7001501269D
:10037000B700950175108100C0050C0901A1018528
:100380000419012AA002150126A002950175108109
:1003900000C005010902A1010901A1000509190117
:1003A000290815002501950875018102050109300C
:1003B00009311581257F9502750881060938158157
:1003C000257F950175088106050C0A3802158125DF
:1003D0007F950175088106C0C005010906A10105C8
:1003E0000719E029E7150025019508750181029597
:1003F00001750881010507190029FF150026FF0076
:1004000095067508810005081901290595057501EE
:100410009102950175039101C00902540003010086
:10042000A0FA0904000001030101000921110100E3
:1004300001224000070581030800010904010001B1
:100440000301020009211101000122470007058272
:100450000308000109040200010300000009211142
:100460000100012232000705830320000112010070
:100470000200000008EF1748600100010200012897
:1004800003500072006F006D006500740068006921
:100490000075006D0020004B006500790062006F60
:1004A00000610072006400000010035000720069D7
:1004B0000079006100640069000000040309042B56
:1004C0000014001A00080015001700290004001687
:1004D00000070009000A00E1001D001B00060019CA
:1004E000000500E000E200E3000A510751B25D1C84
:1004F0000018000C00120013002A000B000D000E63
:10050000000F0034002800110010003600370038BA
:1005100000E500B35D0851AE5DE7004774E40001FB
:10052000000100010000000000000001003400365E
:1005300000370013001C000100040012000800181E
:10054000000C000100380014000D000E001B00011B
:10055000000100010001000100010009000A00067D
:100560000015000F00010007000B00170011001616
:10057000000100050010001A0019001D0001000113
:100580000001000100010001000100010001000163
:1005900000000000000000010014001A0009001310
:1005A000000A0001000400150016001700070001F2
:1005B000001D001B000600190005000100010001DC
:1005C000000100010001000D000F0018001C0034A4
:1005D0000001000B00110008000C00120001000EC9
:1005E0000010003600370038000100010001000152
:1005F00000010001000100010001000100000000F5
:1006000000000001001400070015001A0005000199
:1006100000040016000B0017000A0001001D001B5B
:100620000010000600190001000100010001000196
:100630000001000D00090018001300340001001C27
:10064000001100080012000C0001000E000F00361F
:100650000037003800010001000100010001000125
:100660000001000100010001000000000000000185
:100670000014001A00070009000E00010004001613
:1006800000080017000A0001001D001B00060019E9
:100690000005000100010001000100010001000D42
:1006A00000180015000F00340001001C0011000CA0
:1006B0000012000B00010013001000360037003854
:1006C0000001000100010001000100010001000122
:1006D0000001000100000000000000010000000017
:1006E0000033803F80418001002F80408032804372
:1006F0008031800100348044804580468030800114
:100700000001000100010001000100428036803735
:10071000803D803E80010035803C803880398034C7
:100720000001003B803A80360037003800010001AC
:1007300000010001000100010001000100010001B1
:1007400000000000000000010000005F804B8057A7
:100750008059800100478058804A805B8049800131
:10076000004C805C805D805E80488001000100015B
:10077000000100010001005A804E804F80558056D4
:100780008001004D8054805080518034000100531E
:10079000805280360037003800010001000100015E
:1007A0000001000100010001000100010000000043
:1007B00000000035021E021F022002210222023523
:1007C00000250231002D002E0038002402230231C2
:1007D000022D022E023802010001001B000100015F
:1007E00000010004021E001F002000070201000596
:1007F0000221002200230008020100060224002535
:1008000000260009020100010027483600370033A6
:1008100002010001000100010000000000000000D2
:10082000003A003B003C003D00490039003E003FDB
:1008300000400041004600010042004300440045E2
:10084000004800010001000100010001000100005A
:10085000004B0052004E004B004C00000050005175
:10086000004F004E000100000000004A004D000053
:100870000001000100010001000100010001000170
:10088000000100010000000000000035021E021FF0
:10089000022002210222023500250231002D002E05
:1008A0000038002402230231022D022E02380201F8
:1008B00000010001000100010001002302240225C3
:1008C00002608061800100628026022702360237C2
:1008D00002010063802F0030002F0230020100016E
:1008E00000010001000100330201000100010001CC
:1008F00000000000000000000000000000000000F8
:1009000000000000000000000000000000000000E7
:1009100000000000000000000000000100010001D4
:1009200000010001000100000000000000000000C4
:1009300000000000000000000000000000000000B7
:1009400000000000000000000000000100010001A4
:100950000001000100010001000100010000000091
:10096000000000098017800A8004800D800180103B
:1009700080128002802180158000801180208027D5
:100980008005801E801F801C801D80228001002E1B
:100990008029800E80078014800B800C80138003D8
:1009A000802B8008801680188019802C8006800F8C
:1009B000802D8023801A802A8028800100268025AF
:1009C000801B800100010001000000000000000009
:1009D000001E081F08200821082208290000002BFB
:1009E0000229002B00000000000000AA00A800A9B6
:1009F000002C0000000000000000000000000023A8
:100A000008240825082608270800000000B6000072
:100A100000B700000000002C00AC00AE00AB0000EE
:100A200000000000000000000000000000000001C5
:100A30000001000100000000000000015CA75DB0A3
:100A40005D0000005C00000000B55D0000A85D00D6
:100A500000B45D000000000000A95D00002A5D01F7
:100A600000000000000000000000000000DE5C004C
:100A70000000000000B65D00000000AA5DAF5D0050
:100A8000000000AB5DB15D00000000000000000050
:100A90000000000000000000000100010001000152
:100AA0000000000000000041542B424C45484944DE
:100AB0004D4F555345425554544F4E3D0041542BD4
:100AC000424C454849444D4F5553454D4F56453D81
:100AD00025642C25642C25642C25640041542B426C
:100AE0004C45484944434F4E54524F4C4B45593D59
:100AF0003078253034780041542B424C454B4559D1
:100B0000424F415244434F44453D253032782D30C9
:100B1000302D253032782D253032782D2530327821
:100B20002D253032782D253032782D253032780041
:100B300041542B474150474554434F4E4E0041547A
:100B40002B4556454E54454E41424C453D3078323A
:100B50000041542B4556454E54454E41424C453D6F
:100B6000307831004F4B004154453D300041542B0B
:100B70004741504445564E414D453D50726F6D655D
:100B8000746869756D204B6579626F6172640041AC
:100B9000542B424C45484944454E3D310041542B6D
:100BA000474150494E54455256414C533D31302CEB
:100BB00033302C2C0041545A0041542B424C4550A8
:100BC0004F5745524C4556454C3D2D313200670B31
:100BD0009D0B6D0B8F0BB90BB50B5C2C11241FBE3D
:100BE000CFEFDAE0DEBFCDBF11E0A0E0B1E0E6E09C
:100BF000F7E602C005900D92A238B107D9F724E0BC
:100C0000A2E8B1E001C01D92A23FB207E1F715E0F2
:100C1000CEEED5E004C02197FE010E94962DCD3E78
:100C2000D107C9F70E94880F0C9481330C940000FF
:100C30008F929F92AF92BF92CF92DF92EF92FF92EC
:100C40000F931F93CF93DF93CDB7DEB72A970FB6DD
:100C5000F894DEBF0FBECDBFFC010081D18083813F
:100C60009481892B39F01FEFD11206C091E00F3F1C
:100C700019F403C091E001C090E090FF02C00C9411
:100C8000C10E7F0185E0DE01169601900D928A95D6
:100C9000E1F7F70122818E819F81222349F00E9492
:100CA000FB24182F682F8E819F810E94812503C00D
:100CB0000E945425182F26E3129FF001112436E0DC
:100CC000D39EE00DF11D1124E00FF11DEE0FFF1F6B
:100CD000E154FB4F059114918091A60281FB992765
:100CE00090F990938A0185FB882780F98093890188
:100CF00060918F017091900180919101909192018A
:100D00000E9416148093880180918701909186013A
:100D1000891751F19801225B3D452230310520F1C0
:100D2000F7019281992301F1882369F0809185016F
:100D3000811106C08CE20E94B6268CE20E948526B4
:100D400081E08093850180918601882369F08091FC
:100D50008401811106C08CE20E94B6268CE20E94BA
:100D6000852681E080938401809188018C30C9F4CC
:100D70000B32F2E01F0709F4D5C1C8018D7F8997B6
:100D800009F4D0C10115110509F4CCC1F701828124
:100D9000882321F082EE0E94852603C082EE0E9405
:100DA000B626083AFDE51F0709F457C198F5F70183
:100DB00082810A341105B0F40834110508F06BC1C2
:100DC0000733110509F430C128F40633110509F47D
:100DD000FAC0A8C198012A5331092D30310508F411
:100DE0005AC1A0C1043E110509F4DAC048F4003E1E
:100DF000110509F4D5C0013E110509F4B8C092C12E
:100E0000053E110509F4B3C0073AFDE51F0709F4D3
:100E10001EC188C1003B2DE5120709F464C1F8F436
:100E20000B3A8DE5180709F42EC168F4F7018281A9
:100E3000093AFDE51F0709F41AC10A3A2DE5120720
:100E400009F41BC16FC10E3A3DE5130709F42FC128
:100E50000F3A8DE5180709F065C181E045C1033BF4
:100E60009DE5190709F478C088F4013BFDE51F07EB
:100E700009F43DC1023B2DE5120709F053C125E8F5
:100E800031E046E851E067E871E06CC0043B3DE5C5
:100E9000130709F433C1063B8DE5180709F042C179
:100EA0009FE0909396019093950190939701909372
:100EB00099019093980190939A0190939C0190933B
:100EC0009B0190939D0190939F0110929E0110921F
:100ED000A0019093A2011092A1011092A30110927F
:100EE000A5019093A4011092A6011092A80110925E
:100EF000A7019093A9019093AB019093AA019093BD
:100F0000AC019093B1011092B0011092B201909394
:100F1000B4011092B3019093B5019093B701109270
:100F2000B6011092B8011092BA011092B9019093D3
:100F3000BB011092BD019093BC011092BE011092B2
:100F4000C3019093C2019093C4019093C001909308
:100F5000BF011092C101E3C024E831E047E851E04D
:100F600066E871E0F70182810E94CC14F1C3909190
:100F700088019550923008F0D5C0882329F085E08B
:100F80000E94092686E01CC090918A018091890107
:100F9000981709F4C7C086E00E94092685E010C0B2
:100FA0009091A602292F217092959170882339F093
:100FB000291709F4BBC08DE00E940926B3C08DE05B
:100FC0000E94E425AFC0882309F4C2C380918A013E
:100FD000811105C080918901811104C020C081EE7A
:100FE0000E94852680918901882319F085EE0E9450
:100FF000852683E30E94B62683E30E94852680919E
:101000008A01882319F081EE0E94B6268091890119
:10101000882309F49DC385EE0E94B62699C386E312
:101020000E94B62686E30BC0882309F491C3809101
:10103000A602827239F083E30E94B62683E30E94FF
:10104000852686C387E30E94B62687E3F8CF8823E8
:1010500009F47EC381E090E007C0F7018281882314
:1010600009F476C382E090E00E94341771C38823AC
:1010700009F46EC384E090E0F7CF882309F468C3D5
:1010800088E090E0F1CFF7018281882309F460C302
:1010900080E190E0E9CF81115BC3809188018830C5
:1010A00009F056C3802F0E94B626802FC8CFF701C3
:1010B0008281882389F080918A01811104C0809106
:1010C0008901882321F085E00E94092608C086E076
:1010D0000E94092685E004C085E00E94E42586E0A0
:1010E0000E94E42535C384E08093820202C01092FE
:1010F00082020E943F0F0E944E162AC3F70182818E
:10110000882309F425C3809100018F5F833018F490
:101110008093000102C0109200010E9406150E94F7
:10112000F31516C3F7018281882359F0C801825E46
:101130009C45059730F48EE1800F809382020E94D7
:101140003F0F17FFE6C0F7018281882309F4E1C051
:1011500068010115F0EC1F07F8F020ECD21A90910D
:10116000EF028091F002892B9091F102892B82721B
:10117000BB24B394811101C0B12C0E941A2386951F
:101180008170B81629F0CC0CCD2CCC1CDD08D19484
:10119000E894C7F8DD2402C030E8D31AF601EE0F58
:1011A000FF1FEE0FFF1FE851FF4F85909590A59010
:1011B000B4908114910481E1A806B10408F0A9C09B
:1011C0008114910491E0A906B10428F08091820273
:1011D000823009F49EC00E941A2386958170809304
:1011E0008D010E941A23817080938C01809182026C
:1011F000813039F480918D01882319F089E30E94B0
:101200000F278091F00280938B011092F002809161
:101210008202813071F048F08230C1F0843019F5DB
:1012200086EE0E940F2788E11CC082EE0E94B6263F
:101230001AC083E00E946A2688E10E94B62688E1EF
:101240000E94852683E00E945F260DC080918C015C
:10125000811103C083E50E940F2782EE0E94B6260B
:1012600087E50E940F2781149104E1E0AE06B104E6
:1012700030F180918202811122C0F1E0AF1AB108F1
:10128000D501C40188279C7FAF70BB274AE0B69583
:10129000A795979587954A95D1F7BC01CD017852CE
:1012A0008F4F9F4F0E94040FD501C4019370AA274E
:1012B000BB27BC01CD0174528F4F9F4F02C0C501A7
:1012C000B4010E94040F80918202813059F030F005
:1012D000823089F08430C9F488E215C082EE0E9421
:1012E000852613C08CE20E940F2780918D018823F0
:1012F00061F089E308C082EE0E94852680918C010E
:10130000811103C083E50E940F2780918B01809398
:10131000F002043F2CE5120741F190F4093D8CE501
:101320001807E9F00A3D9CE5190789F1083DECE54D
:101330001E07B1F506E221EE41EE68ED7CE52CC01A
:10134000063FFCE51F07E9F0B0F0073F3CE5130757
:1013500039F507E225EE46EE67EF7CE51DC007E2B2
:1013600025EE45EE69ED7CE517C006E221EE40EE84
:1013700064EF7CE511C007E225EE44EE65EF7CE505
:101380000BC006E221EE42EE66EF7CE505C008E206
:1013900021E045EE6AED7CE5C7010E942623D8C115
:1013A000F7018281882309F45BC110921D03043088
:1013B000FDE51F0758F40B3F2CE5120780F4C80128
:1013C00082509C45449708F035C109C002363DE57E
:1013D000130729F0063A8DE5180709F02BC10E9482
:1013E000891D909394018093930101319CE5190725
:1013F00009F4C6C008F042C00930FCE51F0709F433
:101400009BC000F505303CE5130709F485C078F46E
:1014100003309CE5190709F478C008F07AC002305F
:101420001C4509F0F7C0809193018160F1C007303D
:101430002CE5120709F478C008F07AC08091930176
:101440008061E6C00D308CE5180709F487C058F4B8
:101450000B30ECE51E0709F479C008F07BC08091E1
:10146000930188606FC00F302CE5120709F480C02B
:1014700008F082C080919301877FCAC00E3F8CE53F
:10148000180709F471C000F50531ECE51E0709F4F1
:1014900085C068F403312CE5120709F475C008F023
:1014A00095C00E945426809193018F77B1C00C3F64
:1014B0008CE51807A9F108F054C00B3F1C4509F052
:1014C000A9C08091940140C00230FDE51F0709F4D6
:1014D00089C058F401153DE5130709F45AC008F016
:1014E00069C08091940182602FC002369DE5190782
:1014F00009F47EC0063AEDE51E0709F483C0033007
:101500001D4509F087C060E06EC080919301826044
:101510007FC08091930116C080919301886078C04C
:101520008091940182604FC080919301806270C06D
:101530008091930180646CC00E9454268091930135
:10154000806866C0846064C081603DC08091930102
:101550008E7F5EC0809193018D7F5AC080919301F0
:1015600016C08091940118C0809194018D7F2BC08A
:10157000809193018F7E4CC0809193018F7D48C0F4
:10158000809193018F7B44C080919301877F8B7FF3
:101590003FC0809194018D7F8E7F15C08091930113
:1015A00082FB222720F991E0922790FB82F990FBA1
:1015B00083F92EC080919401982F909591708E7F21
:1015C000892B90FB81F98093940124C00E945426BA
:1015D0008091930187FB222720F991E0922790FBCD
:1015E00087F916C061E08EE090E00E94D23012C010
:1015F0008091930184FB222720F991E0922790FBB0
:1016000084F906C080919301982F909590FB80F902
:1016100080939301609193011091940184E090E094
:101620000E94D230612F82E290E00E94D2300E946C
:1016300054268EC00631FCE51F0759F58091F00253
:101640008A7A91E009F490E090938E01882311F05A
:1016500065E301C069E286EA92E00E94D42216C0E6
:1016600006311C4509F097C080918E01882309F44A
:1016700086C385E3E6EAF2E02CEA32E09281891340
:1016800001C0128231962E173F07C1F70E94121E29
:101690005FC00F3D2CE5120709F446C038F50D3D3B
:1016A0008CE5180709F443C008F046C001151C4535
:1016B00009F071C00E945426EFE7FAE106E0E1501C
:1016C000F0400040E1F700C0000087E797E7909303
:1016D0000108809300089AE088E10FB6F894A89575
:1016E000809360000FBE909360001DC00B35FDE538
:1016F0001F0741F140F40A321D4509F04CC00E9419
:10170000431683E01CC00C358DE51807E9F00D3554
:101710001D4509F040C08091940182FB882780F923
:1017200091E0892712C0FFCF0E949A1D11C00E942C
:101730002E1610921A030CC00E94381682E0809375
:101740001A0306C081E001C080E00E946B1E23C026
:101750008091E602877009F414C3F701828188231F
:1017600009F40FC38091940182FD0BC382E02A9695
:101770000FB6F894DEBF0FBECDBFDF91CF911F91A2
:101780000F91FF90EF90DF90CF90BF90AF909F9020
:101790008F900C944E1EF70182810081D1808823A6
:1017A00059F0802F9D2D0E94FB24182F682F802F29
:1017B0009D2D0E94812505C0802F9D2D0E945425BE
:1017C000182F26E3129FF001112436E0D39EE00D7E
:1017D000F11D1124E00FF11DEE0FFF1FE154FB4F2F
:1017E000859194910E94001C8C01982EF701D28063
:1017F000A580A2943FE0A3228091E6028770B9F011
:10180000DD20A9F0812F807F803421F080E2800FDD
:10181000883068F08091940182FD09C082E00E94C6
:101820004E1E8091E6028770CC24C3948111C12C96
:10183000B12EB2949FE0B9228B2D90E08C309105AF
:1018400008F05EC2FC01EA5AFF4F0C94962D812FDE
:10185000807F1F70882311F01295107FDD20B9F072
:10186000112309F43AC280E2800F883010F0911001
:1018700006C08091F002182B1093F00205C08091F1
:10188000EF02182B1093EF020E94121E26C2802F27
:101890000E948526112309F433C2005E083078F1D6
:1018A000992069F110958091EF0218231093EF02AF
:1018B00029C0812F807F1F70803211F01295107F18
:1018C000992021F0F1E09F16D9F149C0809194014F
:1018D00082FF1BC0DD2069F0112339F08091F002F6
:1018E000182B1093F0020E94121E80E00E94B62670
:1018F00007C280E00E948526112309F401C2812FCE
:101900000E940B1E0E94121EFBC1DD2081F08091FF
:10191000F102AA2051F001E0A01207C0182B1817FD
:1019200009F4EEC11093F102EBC1812B10C0AA2083
:1019300021F021E0A21609F4E3C10E94051E27C090
:10194000DD2041F035E03A1508F4DAC1812F0E941C
:101950007B26D6C184E08A1508F4D2C118C0DD20E8
:1019600049F0AA2099F3F701858180FFB6C18F70F5
:101970008583ECCFAA2059F0093309F0BEC1FFEFEF
:1019800013EF21E0F15010402040E1F7B4C1812F66
:101990000E947426B5C1812F86958695837019F0B3
:1019A000813059F0ADC1DD2019F0C801937002C03B
:1019B00080E090E00E940423ABC1DD2019F0C80153
:1019C000937002C080E090E00E94EE22A1C1812FBE
:1019D000837009F070C0D11097C1902F92959695A1
:1019E0009770990F990F802F8F70882E912CA12CB2
:1019F000B12C092E04C0880C991CAA1CBB1C0A948B
:101A0000D2F704FF12C04FE050E060E070E004C085
:101A1000440F551F661F771F9A95D2F7DB01CA0145
:101A200080959095A095B09503C080E090E0DC0192
:101A300016951695412F4370423019F1A8F5009183
:101A4000F2021091F3022091F4023091F50241303C
:101A500059F088299929AA29BB29BC01CD01602305
:101A60007123822393230AC0082919292A293B2993
:101A7000BC01CD01602B712B822B932B0E942A2657
:101A800043C188299929AA29BB290091F202109102
:101A9000F3022091F4023091F502BC01CD016027E0
:101AA000712782279327EACFBC01CD0168297929C4
:101AB0008A299B29E3CFDD2019F0812F817001C095
:101AC0008695882309F420C1902F9295969597705A
:101AD000990F990F802F8F70882E912CA12CB12CEB
:101AE000092E04C0880C991CAA1CBB1C0A94D2F7AE
:101AF00004FF12C04FE050E060E070E004C0440F0B
:101B0000551F661F771F9A95D2F7DB01CA01809592
:101B10009095A095B09503C080E090E0DC0116950B
:101B20001695412F4370423009F198F500918F01CD
:101B3000109190012091910130919201413059F022
:101B400088299929AA29BB29BC01CD0160237123C9
:101B50008223932324C0082919292A293B29BC015F
:101B6000CD01602B712B822B932B19C088299929C9
:101B7000AA29BB2900918F01109190012091910118
:101B800030919201BC01CD016027712782279327F4
:101B900006C0BC01CD01682979298A299B290E94A8
:101BA000AD25B2C01F70DD2039F0812F0E940926BB
:101BB000802F0E947B26A8C0802F0E947426812F30
:101BC0000E94E425A1C0802F32EF931609F443C090
:101BD000391538F090EF991659F0E1EF9E16B1F1F2
:101BE00077C0F3EF9F16F1F124EF921659F170C010
:101BF000DD2019F134E03A1508F482C01F7181E04C
:101C000090E0A0E0B0E0AC01BD0104C0440F551F5E
:101C1000661F771F1A95D2F780918F0190919001DE
:101C2000A0919101B09192018A019B010827192787
:101C30002A273B27C901B80129C025E02A1508F445
:101C40005FC0DCCF8091940182FF23C0DD2029F0AA
:101C5000812F8F7130C0DD20D9F3812F8F710E94C9
:101C6000E4254EC0DD2079F01F7181E090E0A0E016
:101C7000B0E0BC01CD0104C0660F771F881F991F1B
:101C80001A95D2F703C060E070E0CB010E94AD2549
:101C900037C0DD2099F01F71812F0E9409268091A5
:101CA000940182FD07C038E0139FC00111248360B6
:101CB0008093E602812F0E94092622C081E00E94C3
:101CC0004E1E81E08A15E0F482E00E944E1E18C08C
:101CD000DD2029F0AA2009F4BBCF802F07CEAA204F
:101CE00009F4BBCF893349F49FEFE3EFF1E0915062
:101CF000E040F040E1F700C00000802F0E94852600
:101D000088EF8B0D843020F40E941A230E94141651
:101D1000CC20A9F08091E60280FD11C0F70112826B
:101D20008595859585950E940926C7010E9418060C
:101D30008091E6028595859585950E94E42585E04C
:101D4000F701DE01119601900D928A95E1F78981E4
:101D50009A810E9454259A8106E3809FF001112404
:101D600016E0919FE00DF11D11248981E80FF11D0E
:101D7000EE0FFF1FE154FB4F8591949102C089E261
:101D800079CC2A960FB6F894DEBF0FBECDBFDF9197
:101D9000CF911F910F91FF90EF90DF90CF90BF9068
:101DA000AF909F908F90089580E008959091820267
:101DB000923069F48A3040F490E009966AE070E06D
:101DC0000E946E2D875A01C086500C940F27982FC1
:101DD0009F709A50963010F0805D01C0895A0C9423
:101DE0006614CF93DF93EC010E949C23882341F07B
:101DF000209731F082E08A95F1F700C02197F4CF67
:101E0000CE01DF91CF910895BF92CF92DF92EF92F2
:101E1000FF920F931F93CF93DF936B017C01C7E079
:101E2000D0E00CE110E0BB24B394D701C601002E32
:101E300004C0B695A795979587950A94D2F78F70A9
:101E400029F4B11006C00E94D60E03C00E94D60E1F
:101E5000B12C219704501109CF3F8FEFD80729F0FB
:101E6000C430D10514F7B12CE0CFDF91CF911F9191
:101E70000F91FF90EF90DF90CF90BF900895609109
:101E800082028CE090E00C94D2309091930192FF0A
:101E90000DC0282F2871283019F4877F846006C070
:101EA000282F2471243011F48B7F886093FF0DC09C
:101EB000282F2871283119F4877E846106C0282FC5
:101EC0002471243111F48B7E88612091940120FFCC
:101ED0000DC0382F3871383019F4877F816006C003
:101EE000382F3171313011F48E7F886021FF0DC0A1
:101EF000282F2871283119F4877E816106C0282F88
:101F00002171213111F48E7E886194FD877E0895C0
:101F1000CF93DF93CDB7DEB72A970FB6F894DEBF25
:101F20000FBECDBF84B7877F84BF0FB6F894A89546
:101F300080916000886180936000109260000FBE05
:101F400090E080E80FB6F894809361009093610070
:101F50000FBE85B7806885BF85B7806885BF84ED73
:101F60009EE090938301809382010E94A61A0E94B2
:101F7000C51A8091E20084608093E2007894809199
:101F800095028823A1F01091E9001F709091EC0058
:101F9000892F817090FD80E8182B1092E9008091C4
:101FA000E80083FD0E9492171F701093E90082E001
:101FB00084BD93E095BD9DE797BD80936E0042E29E
:101FC00051E0ACE1B1E061E070E08D91E82FE29585
:101FD000EF70F0E021A18F708B0102C0000F111F84
:101FE0008A95E2F7C801902F9095922391A392A130
:101FF000892B82A34A175B0741F780B3806E80BBB1
:1020000081B38F7181BB45E251E0A2E2B1E061E0B2
:1020100070E08D91E82FE295EF70F0E021A18F70D4
:102020008B0102C0000F111F8A95E2F7C801902FA3
:102030009095922391A392A1892B82A34A175B07C3
:1020400041F783E792E0A1E6B2E0EAE6F2E011921E
:102050001D928E179F07D9F71FEF24E38CE01150D4
:1020600020408040E1F700C0000081E080938202C0
:102070000E943F0FE5E9F1E08EE592E011821082C7
:10208000128233968E179F07C9F78FE08093140250
:102090001092130210921502109211021092100267
:1020A0008093120280930E0210920D0210920F0282
:1020B0000E944E160E9483160E940F170E94F3156D
:1020C0008091E30087FDC3C20E94832A0E944316C9
:1020D00083E080931A0380E090E00E94CC30893E38
:1020E0009E4F11F00E949A1D82E090E00E94C43041
:1020F000809373020E94891D9093940180939301B1
:1021000083E090E00E94C430682F70E080E090E0AF
:102110000E942A268CE090E00E94C43090E0A0E06B
:10212000B0E08093820290938302A0938402B093E4
:1021300085020E94A7230E949923809169008068EC
:1021400080936900EB9ABFEFE3EDF0E3B150E0401C
:10215000F040E1F700C000008FEF0E9450240E9481
:1021600026240E94262484EF0E94502482EE0E949E
:10217000502481E80E9450248AE40E94502489E47B
:102180000E94502482EE0E94502481E80E94502434
:102190008DE40E94502486E00E94502482EE0E942A
:1021A000502481E80E94502480E60E94502481E659
:1021B0000E94502482EE0E9450248CE20E945024FF
:1021C0000E94262480FF0CC082EE0E94502487E4E7
:1021D0000E9450248CE20E94502481E00E945024EE
:1021E00081E091E09093A5028093A402EE24E39411
:1021F000F12C772473945CE3C52ED12C6FE0662E0E
:1022000055245A9472E0472E33E1832E31E0932E09
:1022100001E612E0312CD8019C911C92B8E03B12EF
:102220002FC0E2E2F1E020E030E04191A42FA2953E
:10223000AF70B0E090968C91D8016C914F70D7013F
:1022400002C0AA0FBB1F4A95E2F7AD01482339F43B
:102250008E2D022E01C0880F0A94EAF701C080E09B
:10226000862BD8018C932F5F3F4F23303105E9F641
:10227000981337C080916002882309F45BC046C080
:1022800081B38F71F4012081822B81BBFDE0FA952F
:10229000F1F70000ECE1F1E020E030E04191A42F03
:1022A000A295AF70B0E090968C91D8016C914F7070
:1022B000D70102C0AA0FBB1F4A95E2F7AD01482320
:1022C000C9F48E2D022E01C0880F0A94EAF7862BDE
:1022D000D8018C932F5F3F4F26303105F9F69817C0
:1022E00059F0709260020E94A32290935F02809343
:1022F0005E0202C080E0EBCF33940F5F1F4FBFEF51
:102300008B1A9B0AE9E03E1286CFB4CF80915E0221
:1023100090915F020E949422069760F0AAE6B2E0D4
:10232000E1E6F2E081918D9302E0EA36F007D1F721
:102330001092600280910D0190910E0101968133FF
:1023400015E7910728F490930E0180930D0175C055
:1023500010920E0110920D010E94762B660F771FCE
:10236000881F991F0E94503223E333E343E550E472
:102370000E94073320E030E040E85AE30E94073330
:102380004B015C012DEC3CEC4CE450E40E94AA3182
:1023900087FD21C026E636E646E850E4C501B401D3
:1023A0000E9402331816CCF02DEC3CEC4CE450E4C7
:1023B000C501B4010E943D312CEF3FEF4FE75FE3D1
:1023C0000E94AF3120E030E04FE753E40E94073332
:1023D0000E94213203C060E001C06FEF28E7629FD6
:1023E000C00111246FEF70E00E946E2DCB01B60189
:1023F0000E94822D9B01AC01649EC001659E900DE0
:102400001124B6010E94822D862F2130310531F032
:102410002230310541F48FE090E007C0962D961BE5
:1024200060E08FE002C060E09FE09093AE01809397
:10243000AD016093AF010E94F3150E9483168FB720
:10244000F8944091220350912303609124037091EA
:1024500025038FBFE4E7F2E0AAE6B2E000E010E077
:10246000302F2D919191922721F180E0992493941E
:10247000492F4921D1F089833A83292181E009F448
:1024800080E08B830E94A3228160782F9D838C83C0
:1024900049815A816B818D810E946E13F801EC583D
:1024A000FD4F80819826908218C08F5F990C8630EE
:1024B000F9F60F5F1F4F0930110591F65E825F82BA
:1024C00018860E94A3228160782F9A8789874E817F
:1024D0005F8168858A850E946E138BEE0E9450246E
:1024E0008A3F09F0A7C00E94262480939F020E9481
:1024F00026248093A0020E9426249091A00220917D
:102500009F0291110CC081110AC03091A2023111B9
:1025100006C0309180023227377009F481C02093C1
:102520008002322F307424FF07C031110AC0903866
:1025300041F097FD09C005C0311105C097FF04C0E7
:1025400002C091E801C09FE79093A00225FF07C059
:1025500027FD0AC0803841F087FD09C005C027FD6E
:1025600005C087FF04C002C081E801C08FE7922F39
:10257000977090939F0281958093A10280917F0232
:1025800022FF25C0811108C00E94A32290937E02E1
:1025900080937D0270927F029091A0028091A102AF
:1025A000911102C08823A9F140927F0287FD8F5FBD
:1025B000859581958093A202892F97FD8F5F8595E0
:1025C0008093A3021092A0021092A10222C0813037
:1025D000F1F480917D0290917E020E9494228C32CF
:1025E0009140A8F480919F02846080939F020E9492
:1025F0005917BFEFE0E7F2E0B150E040F040E1F7FB
:1026000000C0000080919F028B7F80939F021092F8
:102610007F0280919F028B7F80939F020E945917B7
:102620001092A0021092A1021092A2021092A30294
:1026300010929F020E941A2390918102891721F023
:10264000809381020E9414160E94ED2ADDCD0E9423
:10265000381682E03ECDE8E8F2E0A491B0E0CD018A
:10266000880F991FA80FB91FAB56BE4F11961C9229
:1026700011971C9212961C92319682E0E83AF80764
:1026800061F7ECE7F2E0A491B0E0CD01880F991F6B
:10269000A80FB91FAB56BE4F11961C9211971C92F2
:1026A00012961C92319682E0E838F80761F7E8E765
:1026B000F2E0A491B0E0CD01880F991FA80FB91FD7
:1026C000AB56BE4F11961C9211971C9212961C92FB
:1026D000319682E0EC37F80761F708951F93CF93A6
:1026E000DF93CDB7DEB767970FB6F894DEBF0FBEA6
:1026F000CDBF4B8B5C8B6D8B7E8B8F8B6111109262
:10270000EF0286E09E01235F3F4FD901E82F1D9223
:10271000EA95E9F795E0FE017396D90101900D92D3
:102720009A95E1F79C894E895F897B897D879E8791
:102730006F87598B488BF901DE01179601900D9236
:102740008A95E1F7CE0107960E941A1F81113EC0BB
:1027500086E0FE013796DE01119601900D928A9572
:10276000E1F7FF81E8856A857B856115710531F0A8
:10277000EF3F31F481E0FF3F19F403C081E001C075
:1027800080E080FD23C02091B40230E0C9010196B1
:10279000877099274091E50250E08417950779F1F9
:1027A000F983EA837D836C8396E0929FD001939FA7
:1027B000B00D1124AB54BD4FFE01319601900D9226
:1027C0009A95E1F78093B4020E94881E16E08091EA
:1027D000E5029091B4028917F9F0189FC001112405
:1027E0008B549D4F0E941A1F8823B1F08091E502FF
:1027F00090E00196877099278093E502E8CF0E94C8
:1028000054261092B4021092E502EEEAF2E086E05D
:10281000DF011D928A95E9F767960FB6F894DEBF3F
:102820000FBECDBFDF91CF911F910895CF92DF9260
:10283000EF92FF926C01EE24FF24C114D104E10455
:10284000F10421F0C701B60120E101C020E0C72E4C
:10285000D82EE92EFF24C114D104E104F10419F0AB
:10286000285FC701B6016B017C0154E0F694E79440
:10287000D794C7945A95D1F7C114D104E104F10457
:1028800019F02C5FC701B6016B017C0142E0F694A0
:10289000E794D794C7944A95D1F7C114D104E104C1
:1028A000F10419F02E5FC701B601DC01CB01B6952A
:1028B000A79597958795892B8A2B8B2B09F02F5FEE
:1028C000822FFF90EF90DF90CF900895DF92EF92EC
:1028D000FF920F931F93CF93DF93E82FF0E0E05226
:1028E000FD4FD490282F26952695269530E0F901A6
:1028F000E053FD4F0491877010E0082E02C015953B
:1029000007950A94E2F701701127F901E054FD4F91
:10291000E490F12C082E02C0F594E7940A94E2F7B3
:1029200091E0E922FF24F901E055FD4FC491D0E088
:1029300002C0D595C7958A95E2F7C170DD270115CC
:10294000110519F081EE0E94B626E114F10419F088
:1029500086EE0E94B6268D2D0E940F27EF2819F0D3
:1029600086EE0E948526012B19F081EE0E948526B5
:10297000CD2B51F08CE2DF91CF911F910F91FF9001
:10298000EF90DF900C940F27DF91CF911F910F9163
:10299000FF90EF90DF9008950F931F93CF93DF93F5
:1029A0008A01E901882381F0C1E0FB01C083FA01BB
:1029B0008081882331F18CE00E94092682EE0E94FA
:1029C000B626C09386021DC0FB011082809186024C
:1029D000882369F082EE0E9485268CE00E94E4251F
:1029E000F801808181110DC0109286020AC0888191
:1029F000811106C08CE20E94B6268CE20E948526D8
:102A00001882DF91CF911F910F910895809100015D
:102A1000813031F018F0823041F108950C942B137D
:102A20000E942B13E8EAF2E087E0A491B0E09D0158
:102A3000220F331FA20FB31FAB56BE4F11968C93BC
:102A400011978C9312968C93319622E0E03BF2071B
:102A500061F78FE0809329021092280210922A02D7
:102A60008093F9011092F80167C0E8E8F2E087E08E
:102A7000A491B0E09D01220F331FA20FB31FAB56EC
:102A8000BE4F11968C9311978C9312968C9331961E
:102A900092E0E83AF90761F7ECE7F2E08FE0A49101
:102AA000B0E09D01220F331FA20FB31FAB56BE4FE4
:102AB00011961C9211978C9312961C92319622E0DB
:102AC000E838F20761F7E8E7F2E08FE0A491B0E0C0
:102AD0009D01220F331FA20FB31FAB56BE4F11969D
:102AE0001C9211971C9212968C93319692E0EC37BF
:102AF000F90761F7E8EAF2E09FE0A491B0E09D01F8
:102B0000220F331FA20FB31FAB56BE4F8FE011969B
:102B10009C9311971C9212961C92319622E0E03BF6
:102B2000F20759F7809329028093280210922A0213
:102B30008093F9018093F8011092FA010895873982
:102B400041F178F4863349F130F4843321F185334F
:102B500031F584E227C08439D1F0863901F581E26C
:102B600021C0843F71F030F4803FD9F0813FB9F447
:102B700081E018C0863F49F030F0873F81F487E05C
:102B800011C084E00FC085E00DC086E00BC080E27C
:102B900009C082E207C083E205C085E203C08FE17D
:102BA00001C080E095E890937A00982F9072906829
:102BB00090937B008F71806480937C0080917A0079
:102BC000806480937A0080917A0086FDFCCF8091AA
:102BD00078002091790090917A009F7790937A0005
:102BE00090E0922B0895259A85B18F7D95B19062E2
:102BF0002FB7F894E5E9F1E032E0EE35F30761F044
:102C0000319148E095B937FF85B9330F000000C016
:102C100085B94A95B9F7F0CF2FBF8FE292E00197BF
:102C2000F1F700C00000089591E0282F227081FF85
:102C300090E080918702981781F090938702222379
:102C400021F08FE08093B10102C01092B101109287
:102C5000B0011092B2010C94F3150895E5E9F1E08A
:102C6000138A128A148A168A158A178A0C94F31505
:102C7000E5E9F1E0138A128A148A8FE0868B858B4E
:102C8000878B0C94F315E5E9F1E0138A128A8FE043
:102C9000848B168A158A178A0C94F3151092960164
:102CA000109295011092970110929901109298013B
:102CB00010929A0110929C0110929B0110929D011A
:102CC00080918202813031F068F0823099F0843056
:102CD000C1F410C08FE0809396018093950180939A
:102CE00097010FC08FE080939901809398018093A2
:102CF0009A0107C08FE080939C0180939B01809391
:102D00009D010C94F3150E9406151092B4011092C7
:102D1000B3011092B5011092B7011092B601109252
:102D2000B8011092BA011092B9011092BB01109231
:102D3000BD011092BC011092BE011092C30110920D
:102D4000C2011092C4011092C0011092BF011092F2
:102D5000C10160918F0170919001809191019091DA
:102D600092010E941614E82F80910F01E81709F4D0
:102D700055C0E0930F01E53010F40C94F3158E2F3D
:102D800090E0FC013597E830F10510F5EE59FF4F62
:102D90000C94962D8FE08093B4018093B501EDCF14
:102DA0008FE08093B701E9CF8FE08093BB01E5CF3F
:102DB0008FE08093BC01E1CF8FE08093C2018093CC
:102DC000C401DBCF8FE08093C0018093BF01D5CFDA
:102DD00087E08093B4018093B3018093B501809321
:102DE000B7018093B6018093B8018093BA018093B4
:102DF000B9018093BB018093BD018093BC01809396
:102E0000BE018093C3018093C2018093C40180936B
:102E1000C0018093BF018093C101AFCF089560913D
:102E2000F2027091F3028091F4029091F5020E94F7
:102E3000161481110AC08FE080939F0110929E01A9
:102E40001092A0011092A20109C010929F0110924D
:102E50009E011092A0018FE08093A2011092A10127
:102E60001092A3010C94F315CF93DF93EC01682F1C
:102E700083E090E00E94D230BE0180E090E00E94AA
:102E80002A26DF91CF910C940F17CF93DF93C2E3E3
:102E9000D0E00E949C23811108C0209731F082E08D
:102EA0008A95F1F700C02197F4CFCE01DF91CF9141
:102EB0000895E091A402F091A502309731F00480CA
:102EC000F581E02D8FE992E009940895EF92FF9249
:102ED0000F931F93CF93DF937C018B010E94892175
:102EE000811119C0E70101151105A1F08091E800D9
:102EF00085FD0AC08091E8008E778093E8000E94EB
:102F00008921882381F307C089918093F1000150C2
:102F10001109E9CF80E0DF91CF911F910F91FF90D0
:102F2000EF9008951F93CF93DF93CDB7DEB7AA97A5
:102F30000FB6F894DEBF0FBECDBFE7E9F2E08FE930
:102F400092E02091F10021938E179F07D1F7809195
:102F50009802833009F463C030F4813071F082301C
:102F600009F49DC0B4C08A3009F489C08B3009F4DB
:102F70006EC0893009F0ABC020C080919702813AC1
:102F800009F0A5C08091E800877F8093E8008091D8
:102F90009B0290919C02892B21F468E08BE892E0DF
:102FA00003C060E080E090E070E00E941022809119
:102FB000E8008B778093E8008AC080919702813285
:102FC00009F085C080919B0290919C02009719F0B6
:102FD000029709F07CC08091E800877F8093E80029
:102FE0008091E80082FD05C0809195028111F8CFA3
:102FF0006EC02091F3008091F20090E0922B029736
:1030000031F48091F100813011F0863021F480910B
:10301000F10080938A028091E8008B7754C0809100
:103020009702813A09F053C080919B0290919C02D3
:10303000892B09F04CC08091E800877F8093E800DD
:103040008091E80080FFFCCF8091100137C0809113
:1030500097028132E1F580919B0290919C02892B2D
:10306000B1F58091E800877F8093E8000E94BC2141
:1030700080919902809310010E94542628C080916B
:103080009702813221F58091E800877F8093E800E4
:103090000E94BC2180919A028093890218C080917D
:1030A0009702813AA1F48091E800877F8093E8003D
:1030B0008091E80080FFFCCF809189028093F1002D
:1030C0008091E8008E778093E8000E94BC21809177
:1030D000E80083FFD9C18091970290919802492F0F
:1030E00050E04A30510508F0CFC1FA01E659FF4FD0
:1030F0000C94962D803821F0823809F0C5C108C0A3
:103100008091930290919402992389F082600FC07C
:1031100080919B028F70873008F0B6C18093E900E0
:103120008091EB0085FB882780F91092E90090914F
:10313000E800977F9093E8008093F1001092F100EF
:103140006FC1282F2D7F09F09FC1882319F082308D
:1031500061F09AC180919902813009F095C1933054
:1031600009F080E0809394022EC080919902811131
:103170002AC080919B028F702FEF280F263008F015
:1031800083C18093E9002091EB0020FF1CC09330A5
:1031900021F48091EB00806214C09091EB0090616B
:1031A0009093EB0021E030E0A90102C0440F551FCD
:1031B0008A95E2F74093EA001092EA008091EB00D2
:1031C00088608093EB001092E9008091E800877F8F
:1031D0008093E8000E94BC2157C1811155C1109114
:1031E00099021F778091E3008078812B8093E30020
:1031F0008091E800877F8093E8000E94BC21809145
:10320000E80080FFFCCF8091E30080688093E300BA
:10321000111102C082E001C083E08093950234C1A5
:103220008058823008F030C12091990230919A0282
:103230002C3D53E0350779F583E08A838AE2898360
:103240004FB7F894DE01139620E03EE051E2E32F01
:10325000F0E050935700E49120FF03C0E295EF7037
:103260003F5FEF708E2F90E0EA3010F0C79601C0FC
:10327000C0968D939D932F5F243149F74FBF809166
:10328000E800877F8093E8006AE270E0CE01019653
:103290000E941022B4C080919B0290919C02432F07
:1032A000552743305105A9F068F44130510509F420
:1032B000FAC04230510509F0E7C084E590E0E9E149
:1032C000F4E04BC04132510529F14232510589F1F8
:1032D000DBC0C901992781309105A1F058F0029710
:1032E00009F0D2C0EFE7F4E0E4918E2F90E0EFE731
:1032F000F4E030C0EBEBF4E0E4918E2F90E0EBEBE8
:10330000F4E028C0E9EAF4E0E4918E2F90E0E9EAE5
:10331000F4E020C08330910508F0B6C0880F991FF3
:10332000FC01E25DFE4F0190F081E02D89E090E02C
:1033300014C08330910508F0A7C0FC01EE0FFF1FF9
:10334000E85DFE4F0190F081E02DDC01AB5DBE4FEA
:103350008C9190E0009709F497C02091E800277FB6
:103360002093E80020919D0230919E022817390792
:1033700008F4C90140E0009789F1209195022223C9
:1033800009F43DC02530D9F12091E80023FD37C074
:103390002091E80022FD2FC02091E80020FFEBCF14
:1033A0004091F3002091F20030E0342B009759F067
:1033B0002830310540F444914093F1003196019753
:1033C0002F5F3F4FF3CF41E02830310509F040E057
:1033D0002091E8002E772093E800CDCF4111CDCF8A
:1033E0000AC080919502882351F0853041F0809188
:1033F000E80083FD04C08091E80082FFF2CF809155
:10340000E8008B778093E8003FC08038E9F5809131
:10341000E800877F8093E800809196028093F10016
:103420008091E8008E77D4CE81112EC080919902D0
:1034300090919A02992702973CF58091E800877F46
:103440008093E80010919902109396020E94BC218B
:10345000111106C08091E30087FD02C081E001C028
:1034600084E08093950242E061EC81E00E94DB21E0
:1034700042E061EC82E00E94DB2142E261EC83E009
:103480000E94DB21809195028091E80083FF10C0AB
:103490008091E800877F8093E8008091EB00806254
:1034A0008093EB0005C082E190E0EDE6F4E055CFBB
:1034B000AA960FB6F894DEBF0FBECDBFDF91CF91B5
:1034C0001F9108951F920F920FB60F9211242F9300
:1034D0003F934F935F936F937F938F939F93AF939C
:1034E000BF93CF93DF93EF93FF93C091E900CF7029
:1034F0008091EC00D82FD17080FDD0E81092E900C7
:103500008091F000877F8093F00078940E9492175A
:103510001092E9008091F00088608093F000CD2B3C
:10352000CF70C093E900FF91EF91DF91CF91BF91F0
:10353000AF919F918F917F916F915F914F913F914B
:103540002F910F900FBE0F901F901895E8EDF0E0AF
:1035500080818E7F80831092E2001092DA001092B8
:10356000E100A0EEB0E08C9181608C9380818F7738
:10357000808319BCA7EDB0E08C918E7F8C93808105
:103580008F7E8083109288020895CF92DF92EF920F
:10359000FF920F931F93CF93DF93C8EDD0E0888104
:1035A0008F7E8883E7EDF0E080818160808384E016
:1035B00082BF81E08093880288818E7F888302EEBB
:1035C00010E0F80110821092DA0081EEC82ED12CA2
:1035D000F601108288818F7788838881806888834C
:1035E00088818F7D888319BC109295021092960273
:1035F000109294021092930290EEE92EF12CF701B2
:1036000080818B7F808388818160888342E060E055
:1036100080E00E94DB21F60180818E7F8083F801AB
:10362000808181608083808188608083F7018081D0
:103630008E7F8083888180618883DF91CF911F9105
:103640000F91FF90EF90DF90CF9008951F920F920F
:103650000FB60F9211242F933F934F935F936F9365
:103660007F938F939F93AF93BF93EF93FF9380913B
:10367000E10082FF09C08091E20082FF05C08091D5
:10368000E1008B7F8093E1008091DA0080FF28C009
:103690008091D80080FF24C08091DA008E7F8093D3
:1036A000DA008091D90019BC80FF16C082E089BD84
:1036B00009B400FEFDCF81E08093950280918802DD
:1036C00081110EC00E94A61A0E94C51A8091E200C4
:1036D00084608093E20004C01092950210928802E8
:1036E0008091E10080FF17C08091E20080FF13C04D
:1036F0008091E2008E7F8093E2008091E200806101
:103700008093E2008091D80080628093D80019BC39
:1037100085E0809395028091E10084FF35C080911F
:10372000E20084FF31C019BC82E089BD09B400FE0B
:10373000FDCF8091D8008F7D8093D8008091E100EB
:103740008F7E8093E1008091E2008F7E8093E20083
:103750008091E20081608093E2008091960288234C
:1037600011F084E007C08091E30087FD02C081E092
:1037700001C083E0809395020E9454260E941A2380
:103780000E941416809195028091E10083FF27C06A
:103790008091E20083FF23C08091E100877F8093C6
:1037A000E10082E080939502109296028091E10000
:1037B0008E7F8093E1008091E2008E7F8093E20013
:1037C0008091E20080618093E20042E060E080E06E
:1037D0000E94DB218091F00088608093F000FF91CF
:1037E000EF91BF91AF919F918F917F916F915F9179
:1037F0004F913F912F910F900FBE0F901F901895F2
:10380000CF93DF938238910569F1B0F4813391054C
:1038100009F46FC048F48932910509F465C08A3211
:10382000910509F46BC08AC08533910509F457C02E
:1038300089339105B9F082C0833E910571F138F466
:10384000803E9105B1F0823E910511F177C0863E30
:103850009105B9F1873E9105C9F1843E910509F0C2
:103860006DC024C02091930120FD53C021FD51C0A3
:1038700065C08091930180FD46C08091940180FFD6
:1038800048C08091930184FD3FC183EE90E03EC12A
:103890008091930182FF3AC0F4CF8091930182FD21
:1038A00035C08091940180FD34C0EBCF80919401AC
:1038B00081FF35C08091930184FD26C187EE90E0A1
:1038C00025C18091930183FF27C0F4CF809193019C
:1038D00083FD22C08091940181FD21C0EBCF8091B6
:1038E000930185FD1FC021C08091930185FD1DC0FE
:1038F00019C08091930186FD1BC01DC0809193016A
:1039000086FD19C015C089E390E000C182EE90E009
:10391000FDC080EE90E0FAC086EE90E0F7C084EE45
:1039200090E0F4C089E290E0F1C085E390E0EEC061
:103930008AE290E0EBC081E390E0E8C0811532E5D7
:10394000930708F069C0811541E5940728F0982F86
:103950008827816F906ADAC0883E910568F5803EBD
:10396000910508F0D3C0883A9105B8F4853A9105DD
:1039700048F0855AE82FF0E0EC5CFE4F808190E043
:103980009064C4C08130910509F4BBC008F4BCC088
:103990008430910508F4B8C0B9C08F3B910508F098
:1039A000B3C0885AE82FF0E0EE0FFF1FE95CFE4F2E
:1039B000808191819464AAC0811520E59207F0F07E
:1039C0009C0174E0369527957A95E1F7922F9370D4
:1039D000482F437021E030E002C0220F331F4A9588
:1039E000E2F73C68392B8F70982F9695969540E2B8
:1039F000949FC0011124822B932B88C0811530E441
:103A0000930718F09F70906A81C09C013A95211528
:103A10003F4108F47BC078C0EC01C11586E5D807AA
:103A2000E8F5C11525E5D20748F08C2F0E94450F17
:103A30008F7190E0982F8827906268C0C11534E597
:103A4000D30728F09C2F8827846F906A5FC0AE014F
:103A5000437055272C2F26952695C115D34578F40C
:103A600081E090E002C0880F991F4A95E2F740E29A
:103A7000249F90011124822B932B9C6847C081E0E6
:103A800090E002C0880F991F4A95E2F740E2249F18
:103A900090011124822B932B9A6838C0C1152AE516
:103AA000D207F8F4C11539E5D30790F08C2F8F7049
:103AB0000E94450F94E0D695C7959A95E1F7CF708F
:103AC000D0E0DC2FCC27D0699E01282BC9011EC075
:103AD000C11548E5D407C0F09C2F8827806F906AF5
:103AE00015C0CE0190568115904270F48D2F8F71C4
:103AF0000E94450F282F2F71CE0199279062922B9B
:103B000005C081E090E002C080E090E0DF91CF91BD
:103B10000895CF9384E090E00E94C430C82F82E2E1
:103B200090E00E94C4302C2F30E0A901582BCA012C
:103B3000CF91089569EE7EEF80E090E00E94F03032
:103B400060E082E090E00E94D23060E083E090E0AC
:103B50000E94D2301092F2021092F3021092F402FC
:103B60001092F50260E084E090E00E94D23060E0C4
:103B700082E290E00E94D23060E085E090E00E9416
:103B8000D23060E086E090E00E94D2306FEF87E0B4
:103B900090E00E94D23040E050E0BA0188E090E02E
:103BA0000E94E43060E08DE090E00E94D23040E07E
:103BB00050E0BA0188E190E00E94E43060E087E1E3
:103BC00090E00E94D23040E050E0BA018CE190E0F9
:103BD0000E94E43060E070E080E290E00E94F0300B
:103BE00040E050E0BA0188E190E00E94E43040E01B
:103BF00050E0BA018FE090E00E94E43040E050E0F5
:103C0000BA0183E190E00C94E4308091F1028111DB
:103C10001092F102089580959091F002892380938B
:103C2000F00208959091F0028091EF02982B90930A
:103C3000A6028091F102882389F0892B8093A60245
:103C4000E8EAF2E097E080E0915029F02191222308
:103C5000D9F38F5FF9CF81110E94051E48E050E033
:103C600067EE72E086EA92E00E947433892BA9F035
:103C700088E0E6EAF2E0A7EEB2E001900D928A95C4
:103C8000E1F7E091A402F091A502309731F00280B3
:103C9000F381E02D86EA92E0099408952091E602EE
:103CA000809582238093E602982F977099F430E0F4
:103CB000482F082E000C550B2417350759F090910A
:103CC000940192FD07C08595859585950E94E42510
:103CD0001092E6020895CF93C0919401C2FB9927F8
:103CE00090F9981799F080FBC2F9C0939401609104
:103CF000930184E090E00E94D2306C2F82E290E049
:103D00000E94D23082E0CF910C944E1ECF91089544
:103D10008091E5029091B402891719F08F5F877046
:103D2000FBCF08950F931F93CF93DF938091B3023E
:103D300082958F7009F05DC08091B002882309F4EC
:103D400058C08091E5021091B4026091AE0270916A
:103D5000AF02C091B102D091B20291E06F3F09F081
:103D600090E0292F06E0811709F443C0209721F045
:103D70007F3F21F030E003C031E001C0322F90E0FE
:103D800030FD34C0089FF001099FF00D1124DF01C0
:103D9000AB54BD4F11963C911197371327C03C91FE
:103DA000361324C012963C91129731111FC01396FE
:103DB0004D915C9114974C1B5D0B483C5105B0F440
:103DC0008091B3028F7080618093B302E654FD4FFF
:103DD00080818F70806180838EEA92E00E94180655
:103DE000DF91CF911F910F910C94881E01968770DF
:103DF000BACFDF91CF911F910F910895CF93DF93A9
:103E0000EC010E94FB2426E3829FC0011124FC01E7
:103E100026E0D29FE00DF11D1124EC0FF11DEE0FF5
:103E2000FF1FE154FB4F859194910E94001CDF918C
:103E3000CF9108959F92AF92BF92CF92DF92EF926F
:103E4000FF920F931F93CF93DF93CDB7DEB76197A8
:103E50000FB6F894DEBF0FBECDBF8C0185E0F80130
:103E6000DE011D9601900D928A95E1F7F801E2803E
:103E70009091AE026091AF024091B1025091B202B6
:103E80004115510531F06F3F31F481E09F3F19F446
:103E900003C081E001C080E0F82FF1709F2E80FD0B
:103EA0001AC1F80130812181C380D4808EEAA82E06
:103EB00082E0B82EF090B002F601E41BF50BFF2073
:103EC00009F4C6C08091B302E83CF10508F091C046
:103ED000482F407F09F050C0621311C093130FC0E8
:103EE000FE2CE1100CC08F7080618093B302C5017D
:103EF0000E9418068091B302F801858329C1CD285C
:103F000031F02F3F31F481E03F3F19F403C081E0ED
:103F100001C080E080FD03C081E08E2502C080E00A
:103F200090E0F82FF170FF2E80FF1CC08091E50219
:103F30004091B40256E0841709F4E8C090E0589F1D
:103F4000F001599FF00D1124EB54FD4F61812613B0
:103F500006C06081631303C06281E61203C001964C
:103F60008770E9CFFE2CEE2009F4F2C08091B302F5
:103F700081608093B30249C0621306C0931304C0EA
:103F8000E11002C0F80186C0C8010E9434268823CF
:103F900051F1EE2041F12091B302822F82958F7072
:103FA00090E0029774F08091AE029091AF029887F2
:103FB0008F831986DB86CA862C87CE0107960E94DE
:103FC000180686E0F801AEEAB2E001900D928A95FB
:103FD000E1F70E94921E0AC06217C9F0C8010E9450
:103FE000342681111EC0C8010E941806FF24F394D4
:103FF000AFC0482F407F81F78EEA92E00E941806FA
:1040000086E0F50111928A95E9F7F12CA1C093138E
:10401000E5CFE110E3CFF8018583C8010E941806BF
:1040200054C0EE2001F32091B302822F82958F704D
:1040300090E0029734F28091AE029091AF029A83A1
:1040400089831B82DD82CC822E83CE010196B7CF7D
:10405000E83CF105D0F5FE2CEE2029F2621327C0D2
:10406000931325C02091B30220FD18C0822F8295A2
:104070008F70482F50E04115510581F0F8012583DC
:104080004F30510541F08F5F982F9295907F822F8E
:104090008F70892B8583C8010E94180686E0F8017D
:1040A000AEEAB2E001900D928A95E1F751C0C801E5
:1040B0000E943426811185CF8091B3028160809364
:1040C000B302C8010E94180643C086E0F5011192B0
:1040D0008A95E9F73DC0EE2009F485CFC8010E941A
:1040E0003426F82E882309F47ECF86E0F801AEEA64
:1040F000B2E001900D928A95E1F78091AE02909125
:10410000AF020E94FE1E0E94921E22C03D872E8793
:104110008D859E850E94FE1E292F22952F702230AC
:1041200028F49F7039F0811105C00BC0243028F4A9
:104130009F7049F4805E883020F0C8010E94180604
:104140009F2CF92C05C0F8019581907F99F7F9CF44
:104150008F2D61960FB6F894DEBF0FBECDBFDF91F5
:10416000CF911F910F91FF90EF90DF90CF90BF9074
:10417000AF909F900895089580918A0208955A986B
:10418000529A089552985A9A82E08A95F1F700C09F
:1041900089B182FB882780F9089580932603709364
:1041A00028036093270380919502843001F583E012
:1041B0008093E9008FEF9091E800815095FD06C053
:1041C0009AE69A95F1F700C08111F5CF8091E80049
:1041D00085FF0DC040E050E063E070E086E293E0D0
:1041E0000E9466178091E8008E778093E80008951A
:1041F000BC0183E00C94CD2080911A03811109C089
:104200008091E30087FD04C00E94832A83E0089523
:1042100082E00895CF93DF93EC010E94FC2083306D
:1042200029F4CE01DF91CF910C940D2CBE0184E0D6
:10423000DF91CF910C94CD200F93CF93DF93EC01BE
:104240000E94FC20833041F408812C814B816A81DB
:1042500089810E94322C1FC082E08093E9008FEF99
:104260009091E800815095FD06C09AE69A95F1F785
:1042700000C08111F5CF8091E80085FF0CC040E0BF
:1042800050E065E070E0CE010E9466178091E80082
:104290008E778093E800DF91CF910F910895CF93AF
:1042A000DF93EC010E94FC20833049F4BE016E5F75
:1042B0007F4F46E08881DF91CF910C94AD2B81E058
:1042C0008093E9008FEF9091E800815095FD06C042
:1042D0009AE69A95F1F700C08111F5CF8091E80038
:1042E00085FF14C040E050E068E070E0CE010E941D
:1042F00066178091E8008E778093E80088E0FE01E1
:10430000ABE8B2E001900D928A95E1F7DF91CF9191
:1043100008952091E4003091E50095E64091EC008D
:10432000842F817040FF23C08091E80080FD1DC074
:1043300080919502882399F0853099F08091EB0067
:1043400085FD11C04091E4005091E5002417350728
:1043500029F3915011F09A01E1CF84E0089582E0B1
:10436000089583E0089581E0089580E008954091E4
:10437000E80042FFDDCF08958091970287FF11C0CA
:104380008091E80082FD05C0809195028111F8CFEF
:1043900011C08091E8008B770BC080919502882333
:1043A00049F08091E80080FFF8CF8091E8008E7797
:1043B0008093E8000895982F973068F59093E9006E
:1043C000981739F07091EC002091ED005091F000B9
:1043D00003C0242F762F50E021FD02C09F5FECCF59
:1043E0003091EB003E7F3093EB003091ED003D7F4C
:1043F0003093ED003091EB0031603093EB0070931F
:10440000EC002093ED005093F0002091EE0027FD8A
:10441000E5CF80E008958F708093E90081E00895F2
:1044200020919D0230919E022617370748F06115B2
:10443000710539F42091E8002E772093E80001C03F
:10444000B901FC0120E06115710579F180919502B7
:104450008823F1F18530F1F18091E80083FD3CC0C3
:104460008091E80082FD2EC08091E80080FFEBCFB4
:104470002091F3008091F20090E0922B611571057C
:1044800051F08830910538F421912093F10061506A
:1044900071090196F3CF21E0089709F020E080919F
:1044A000E8008E778093E800CECF2111CFCF0AC0ED
:1044B00080919502882361F0853061F08091E80059
:1044C00083FD0AC08091E80082FFF2CF80E008956A
:1044D00082E0089583E0089581E0089578941F9222
:1044E0000F920FB60F9211248F939F93AF93BF93A8
:1044F0008091220390912303A0912403B09125037E
:104500000196A11DB11D8093220390932303A093D4
:104510002403B0932503BF91AF919F918F910F908A
:104520000FBE0F901F9018959C014FB7F894809183
:10453000220390912303A0912403B09125034FBF40
:10454000821B930B08952FB7F894809122039091CA
:104550002303A0912403B09125032FBF08951F9238
:104560000F920FB60F9211248F939F93AF93BF9327
:104570008091220390912303A0912403B0912503FD
:104580004196A11DB11D8093220390932303A09314
:104590002403B0932503BF91AF919F918F910F900A
:1045A0000FBE0F901F9018959C01FC0132969FEF53
:1045B00080E04191461789F09F3F19F4411101C0F5
:1045C000982F8F5F8630A9F79F3F39F0F901E90FE7
:1045D000F11D97FDFA9562830895089520912003B7
:1045E000309121032817390771F0909321038093AC
:1045F0002003E091A402F091A502309721F00084FD
:10460000F185E02D0994089520911E0330911F0338
:104610002817390771F090931F0380931E03E091D0
:10462000A402F091A502309721F00680F781E02DD9
:1046300009940895E091A402F091A502309721F029
:104640000190F081E02D099480E008950F931F936D
:10465000CF93DF93C42FD22FFC0182818823C9F02E
:1046600040931D030E94A32290931C0380931B037D
:1046700080E28C0F883008F057C0C77081E001C01D
:10468000880FCA95EAF7DF91CF911F910F910C9493
:104690007B2680911D03481330C080911B039091AD
:1046A0001C030E949422883C910538F510E21D0FEE
:1046B000CD17B9F080E28C0F883040F4C77081E0EC
:1046C00001C0880FCA95EAF70E947426183028F5B1
:1046D00081E09D2F977001C0880F9A95EAF70E949C
:1046E0007B26802F0E940F271830F0F4D77081E0CE
:1046F00001C0880FDA95EAF70AC080E28C0F883093
:1047000098F4C77081E001C0880FCA95EAF7DF917D
:10471000CF911F910F910C947426802FDF91CF9130
:104720001F910F910C940F27DF91CF911F910F9143
:10473000089552985A9A089553985B9A82E08A9500
:10474000F1F700C089B183FB882780F90895539859
:104750005B9A08951F920F920FB60F9211242F9318
:104760003F934F935F936F937F938F939F93AF93F9
:10477000BF93EF93FF930E949C23811156C08091B9
:1047800019038F5F809319038A3028F4823068F40C
:10479000813031F043C08A30D1F08B3021F13EC0FE
:1047A0000E94C22081113AC040C0809118038695B2
:1047B000809318030E94C2208823B9F180911803C6
:1047C000806880931803809111018F5F2CC00E9434
:1047D000C22090911101882319F090FF1FC025C0BD
:1047E00090FD1CC022C00E94C2208823B9F05091C5
:1047F00018034FB7F8948091170390E09C012F5F46
:104800003F4F2F71332760911603621731F0FC017F
:10481000EA50FD4F5083209317034FBF10921903A6
:104820001092180381E080931101FF91EF91BF91E5
:10483000AF919F918F917F916F915F914F913F9138
:104840002F910F900FBE0F901F9018958AE1815005
:1048500051F49FB7F89420911603809117038213A7
:1048600012C080E01BC03FB7F894209117039091CD
:1048700016033FBF2913EDCFEFECF7E03197F1F7C7
:1048800000C00000E4CF30E0F901EA50FD4F808124
:104890002F5F3F4F2F713327209316039FBF08953B
:1048A000EF92FF920F931F93CF93DF93E82EEB9835
:1048B0005B98539A0E94992387EC90E00197F1F757
:1048C00000C000000E94BF200E94A72380E197E261
:1048D0000E94F10E892B09F475C0C0E0D0E011E010
:1048E000F12C01E0C7010C2E02C0959587950A9422
:1048F000E2F780FF04C010270E94992302C00E94A3
:10490000BF200E944517892B09F45CC082E390E028
:104910000E94F10E892B09F455C02196C830D105AB
:1049200009F788E28A95F1F7112319F00E9499237B
:1049300002C00E94BF200E944517892B09F442C083
:1049400082E390E00E94F10E892BE1F198E29A95C2
:10495000F1F70E949923C2E3D0E00E94C22088238D
:1049600041F0209779F122E02A95F1F700C02197D4
:10497000F4CFCD2B39F182E390E00E94F10E892B28
:1049800009F10E944517892BE9F0C2E3D0E00E94AB
:10499000C220811108C02097A9F082E08A95F1F722
:1049A00000C02197F4CFCD2B69F00E94A7230E946D
:1049B0009923EB9ADF91CF911F910F91FF90EF9088
:1049C0000C9426240E94A7230E949923EB9A80E04E
:1049D000DF91CF911F910F91FF90EF90089580E0AC
:1049E00090E00E94042380E090E00E94EE2210926A
:1049F000EF020C94121E8F929F92AF92BF92DF92A1
:104A0000EF92FF920F931F93CF93DF9380908F01CC
:104A100090909001A0909101B09092014091F2028B
:104A20005091F3026091F4027091F502842A952A64
:104A3000A62AB72ACFE1D0E026E0929F7001112488
:104A400096E3D92E082F10E0D501C4010C2E04C026
:104A5000B695A795979587950A94D2F780FD04C0DF
:104A6000219790F780E014C0DC9EF001DD9EF00DF0
:104A70001124EE0DFF1DE00FF11FEE0FFF1FE1549B
:104A8000FB4F859194910E94001C019749F38C2F54
:104A9000DF91CF911F910F91FF90EF90DF90BF902A
:104AA000AF909F908F900895292F220F920F990F0A
:104AB000890F682F669566956695982F977085E0A3
:104AC000689FB001112440E050E080E0FB01E40F5A
:104AD000F51FE75DFC4F208130E0092E02C03695BE
:104AE00027950A94E2F721703327042E01C0220F84
:104AF0000A94EAF7822B4F5F5F4F4530510531F73B
:104B00000895292F220F920F990F890FE82FE6950C
:104B1000E695E695877051E001C0550F8A95EAF752
:104B200085E0E89FF0011124E75DFC4F20E030E0D4
:104B300070E04081CB01022E02C0969587950A94C1
:104B4000E2F78170819584278523842781932F5FE5
:104B50003F4F2530310569F708950F931F938B015F
:104B60009C010078117022273327DC01CB0100382B
:104B700011402105310511F4926001C09D7F8C0127
:104B80009D01007214702227332700321440210542
:104B9000310559F08C019D010074147022273327D0
:104BA000003414402105310511F4986001C0977F4D
:104BB00080938F0190939001A0939101B093920103
:104BC0001F910F910C94EF240F931F9341E050E03D
:104BD00060E070E004C0440F551F661F771F8A9580
:104BE000D2F7409550956095709580918F01909186
:104BF0009001A0919101B09192018A019B0108233B
:104C000019232A233B23C901B8011F910F910C944A
:104C1000AD250F931F9341E050E060E070E004C0C9
:104C2000440F551F661F771F8A95D2F780918F0119
:104C300090919001A0919101B09192018A019B0104
:104C4000082B192B2A2B3B2BC901B8011F910F915F
:104C50000C94AD256093F2027093F3028093F402FA
:104C60009093F5020C94EF24FC01808191810E94C5
:104C7000FE1E92959F70963079F010F4925001C00C
:104C80009A50923068F4803F69F018F4883E40F4FE
:104C900009C0843F29F406C0883E20F0813F11F00E
:104CA00080E0089581E008951092F00286E0E8EA3D
:104CB000F2E0DF011D928A95E9F70C94EF24882336
:104CC00041F080959091EF0289238093EF020C943C
:104CD000121E0895882339F09091EF02892B80935A
:104CE000EF020C94121E0895882321F00E940B1EDF
:104CF0000C94121E0895882339F09091F002892BAC
:104D00008093F0020C94121E0895882371F19CEF99
:104D1000980F913A60F4E6EAF2E09281891301C0BB
:104D20001282319692E0EC3AF907B9F70DC090E2A1
:104D3000980F983058F4982F977081E001C0880F31
:104D40009A95EAF70E940B1E0C94121E9BE5980F91
:104D5000933020F480E090E00C940423885A87314B
:104D600020F480E090E00C94EE220895CF93882305
:104D700009F453C09CEF980F913AF8F4C82FE8EA71
:104D8000F2E08EEA92E02191C21721F08E179F0780
:104D9000D1F70DC0E6EAF2E08281C81301C01282A9
:104DA000319642E0EC3AF407B9F70E94121E6C2FDC
:104DB00086EA92E00E94D42213C090E2980F9830C5
:104DC00090F4877021E030E0A90102C0440F551F24
:104DD0008A95E2F7CA019091F002892B8093F00244
:104DE000CF910C94121EEBE5E80FE33040F4F0E0B5
:104DF000EC5CFE4F808190E0CF910C940423885AA4
:104E0000873158F4E82FF0E0EE0FFF1FE95CFE4F0A
:104E100080819181CF910C94EE22CF9108951F93C0
:104E2000CF93DF93182F893319F0C0E0D0E002C090
:104E3000C0E5D0E0812F0E94B626209741F08FEC8C
:104E400097E00197F1F700C000002197F6CF812F7E
:104E5000DF91CF911F910C948526EF92FF920F93D3
:104E60001F93CF93DF93EC018B0122E030E040E011
:104E700060E084E30E946D2C0E94A3227C01888163
:104E80000E94E62C8E3F9105A9F40E94462D82E4F3
:104E90008A95F1F700C022E030E040E060E084E372
:104EA0000E946D2CC7010E9494228017910738F34D
:104EB000C0E00AC06B816F7770E06D5F7F4FCE01FD
:104EC00001960E94162DC1E00E94462D8C2FDF9185
:104ED000CF911F910F91FF90EF900895EF92FF9265
:104EE0000F931F93CF93DF93EC017B010E94A322CA
:104EF0008C0166990CC082E08A95F1F700C0C80168
:104F00000E9494228E159F05A0F3C0E035C022E0D8
:104F100030E040E060E084E30E946D2C0E94FE2CB3
:104F200088838E5F8230A8F40E94462D82E48A95A1
:104F3000F1F700C022E030E040E060E084E30E944E
:104F40006D2CC8010E9494228E159F0538F3C0E095
:104F500011C063E070E0CE0101960E942E2D6B819E
:104F60006F7770E06131710524F4CE0104960E94E0
:104F70002E2DC1E00E94462D8C2FDF91CF911F91E5
:104F80000F91FF90EF9008951F93CF93DF93CDB7CC
:104F9000DEB764970FB6F894DEBF0FBECDBFE091C9
:104FA000510390915003E91709F43FC0182F669BF5
:104FB00021C066E970E0CE0101960E946E27882329
:104FC000A1F18C8187FD0DC0209151038091500388
:104FD000281759F130E02F5F3F4F2170332720937E
:104FE0005103112311F190915103809150039813B3
:104FF0001AC01BC0F0E0EE0FFF1FE45BFC4F808186
:1050000091810E9494228D32914078F080915103D9
:1050100090915003891749F090E00196817099278B
:105020008093510302C06699C4CF64960FB6F8947A
:10503000DEBF0FBECDBFDF91CF911F9108956F925C
:105040007F928F929F92AF92BF92CF92DF92EF9218
:10505000FF920F931F93CF93DF93CDB7DEB7A8973F
:105060000FB6F894DEBF0FBECDBF7C018B016A0185
:105070004901FC0101900020E9F7CF0101975C0193
:10508000672B61F09091500380915103981721F0A4
:1050900081E00E94C427F6CFF801108240E1742E0F
:1050A0005AE0652EA5014E195F09888D41315105E1
:1050B000DCF07D8A1E8A6F8A807880618068888FA4
:1050C000F701DE015996872D01900D928A95E1F73F
:1050D000B401CE0145960E942D27882309F464C0AF
:1050E000F0E1EF0EF11CDECF80E18D8B1E8A8AE0AD
:1050F0008F8B842F8F77888F5527B701CE014996E4
:105100000E94DC2DB401CE0145960E942D27F82E79
:10511000882309F449C001151105E1F40E94A32276
:105120008C018091500390E09C012F5F3F4F2170D4
:10513000332740915103421709F45AC0880F991F31
:10514000FC01E45BFC4F11830083209350030E9419
:10515000A32252C05801AC0CBD1C78016CE271E076
:10516000CE0101960E946E278823F1F0898180325A
:1051700019F0F801108218C08C818F77CA2CCE18D4
:105180008C1508F4C82ECC2051F0D12CA601BE01FC
:105190006B5F7F4FC7010E94DC2DEC0CFD1C8C81E6
:1051A00087FDDCCFF70106C0F12C26C07F0180818E
:1051B0008A3039F41082F70131970E171F07B0F3C8
:1051C00002C08D30B9F36AE070E0C8010E94F02D92
:1051D000009719F08C010F5F1F4F64E67BE0C80158
:1051E0000E94C32D21E0892B09F020E0F22E04C09B
:1051F00080E00E94C42795CF8F2DA8960FB6F89413
:10520000DEBF0FBECDBFDF91CF911F910F91FF90F9
:10521000EF90DF90CF90BF90AF909F908F907F9056
:105220006F9008958F929F92AF92BF92CF92DF922C
:10523000EF92FF920F931F93CF93DF93CDB7DEB71B
:105240007C015B014A01CDB6DEB60E94D32D0196EA
:105250002DB73EB7281B390B0FB6F8943EBF0FBED3
:105260002DBF0DB71EB70F5F1F4FB701C8010E94BA
:10527000CC2D26E930E0A401B501C8010E941F2809
:105280000FB6F894DEBE0FBECDBEDF91CF911F9159
:105290000F91FF90EF90DF90CF90BF90AF909F90D5
:1052A0008F9008958F929F92AF92BF92CF92DF928C
:1052B000EF92FF920F931F93CF93DF93CDB7DEB79B
:1052C000CA57D1090FB6F894DEBF0FBECDBF7C011F
:1052D0009091500380915103981301C19091E30480
:1052E0008091E204981709F4FAC08AE0899F90013E
:1052F00011242E5A3C4FF901DE01AF58BF4F0190E7
:105300000D928A95E1F7F901C08015810681D78059
:10531000908481840E94A3229093EF048093EE04F2
:10532000F1E0CF1679F1CF1628F022E0C21609F489
:1053300052C0BAC067EF7AE0CE0101965C010E94CC
:10534000CC2D1F928F921F929F921F92DF921F92DD
:105350000F931F921F93E6968FADE6971F928F9340
:10536000E5968FADE5971F928F93BF92AF921F92F4
:1053700080E38F938E010F5B1F4F1F930F930E944B
:10538000032E1BC06CED7AE08E010F5F1F4FC8012A
:105390000E94CC2DE6968FADE6978F93E5968FAD64
:1053A000E5978F931F930F931F9280E38F93005C79
:1053B0001F4F1F930F930E94032E970140E050E070
:1053C00060E070E0C8010E941F280FB6F894DEBFAD
:1053D0000FBECDBF67C06DEB7AE0CE0101965C01D8
:1053E0000E94CC2D802F002E000C990B9F930F93C1
:1053F000812F012E000C990B9F931F93E6968FAD82
:10540000E697282F082E000C330B3F938F93E596D9
:105410008FADE597282F082E000C330B3F938F9309
:10542000BF92AF921F9280E38F938E010F5B1F4F4D
:105430001F930F930E94032E970140E050E060E01D
:1054400070E0C8010E941F280FB6F894DEBF0FBE9F
:10545000CDBF8823C1F167EA7AE0C8010E94CC2D54
:10546000D0FE05C065E671E0C8010E94E52DD1FEC1
:1054700005C067E671E0C8010E94E52DD2FE03C0B9
:1054800069E671E004C0D11005C06BE671E0C801A7
:105490000E94E52D970140E050E060E070E0C80117
:1054A0000E941F28882379F08091E3049091E20400
:1054B0008917A9F090E0019668E270E00E946E2DD5
:1054C0008093E3040CC0FFE729EA33E0F150204069
:1054D0003040E1F700C0000081E00E94C427C658B8
:1054E000DF4F0FB6F894DEBF0FBECDBFDF91CF9177
:1054F0001F910F91FF90EF90DF90CF90BF90AF90F2
:105500009F908F9008958091E40408950F931F93C6
:10551000CF93DF93CDB7DEB7C258D1090FB6F89459
:10552000DEBF0FBECDBF8091E50481111EC0109279
:10553000E6041092E4046E9876980E94652C549AC2
:105540005C9A5C988FE19EE40197F1F700C000003F
:105550005C9A9FEF29E688E1915020408040E1F776
:1055600000C0000081E08093E5041092E6040EEC98
:105570001BE042E050E0B801CE018F579F4F0E94E0
:10558000BA2D40E850E0BE016F5F7F4FCF57DF4F2D
:1055900088819981C158D0400E941229882379F0CE
:1055A0000E5F1F4F9BE00A3D190719F781E08093BA
:1055B000E6040E94A3229093EF048093EE0480916E
:1055C000E604CE57DF4F0FB6F894DEBF0FBECDBF57
:1055D000DF91CF911F910F910895CF93DF93CDB7B6
:1055E000DEB7E0970FB6F894DEBF0FBECDBF809157
:1055F000E604811105C00E94862A882309F46DC043
:1056000081E00E94C4278AE090E00E9452298091A4
:10561000EE049091EF040E949422893E9340C8F1D9
:105620008091E704811117C040E350E0BE016F5F35
:105630007F4F81E59BE00E941229882349F040E3D7
:1056400050E0BE016F5F7F4F8EE39BE00E94122906
:1056500081E08093E7040E94A3229093EF0480935B
:10566000EE0440E350E0BE016F5F7F4F80E39BE0BC
:105670000E941229882369F0CE0101960E949C2D78
:1056800021E0892B09F420E08091E4048213209327
:10569000E4048091E8049091E9040E94942281310D
:1056A0009742D8F09091500380915103981315C000
:1056B0000E94A3229093E9048093E80485E30E946A
:1056C0009F15092E000CAA0BBB0B8093EA04909344
:1056D000EB04A093EC04B093ED04E0960FB6F894BD
:1056E000DEBF0FBECDBFDF91CF9108956091EA0478
:1056F0007091EB048091EC049091ED0408950F9368
:105700001F93CF93DF93EC01FB018C0100571E4FD9
:10571000D8012C9130E0C901019668E270E00E9446
:105720006E2DDE01AF56BE4F9C91981781F09AE026
:10573000929FD001939FB00D1124AC0FBD1F01901B
:105740000D929A95E1F7F801808381E001C080E035
:10575000DF91CF911F910F910895FF920F931F93A7
:10576000CF93DF93CDB7DEB72A970FB6F894DEBF9D
:105770000FBECDBF8B01F42E19828C830E94A32211
:105780009B838A83F80180818D83FF2011F08181C2
:1057900001C080E08E83F1E0FF1518F4F8018281EA
:1057A00001C080E08F83F2E0FF1518F4F8018381D7
:1057B00001C080E08887F3E0FF1518F4F8018481C8
:1057C00001C080E08987F4E0FF1518F4F8018581B5
:1057D00001C080E08A87BE016F5F7F4F82E593E062
:1057E0000E947F2B811105C086E990E00E9452291A
:1057F000C9CFF6E0FF1528F48AEFF80E0A5F1F4FB5
:10580000C1CF2A960FB6F894DEBF0FBECDBFDF9191
:10581000CF911F910F91FF900895CF93DF93CDB754
:10582000DEB72A970FB6F894DEBF0FBECDBF21E0DA
:1058300029839D838C83BE016F5F7F4F82E593E058
:105840000E947F2B811105C086E990E00E945229B9
:10585000F2CF2A960FB6F894DEBF0FBECDBFDF9110
:10586000CF9108950F93CF93DF93CDB7DEB72A97EB
:105870000FB6F894DEBF0FBECDBF92E099838C8344
:105880006D834E832F830887BE016F5F7F4F82E554
:1058900093E00E947F2B811105C086E990E00E9471
:1058A0005229F2CF2A960FB6F894DEBF0FBECDBFB5
:1058B000DF91CF910F9108951092E2041092E304CA
:1058C000ECE4F3E0148215820895289A219A229A32
:1058D00023982B9880E58CBD0895909112019F3FED
:1058E00009F072C08F3F09F46FC0611103C01092BC
:1058F000F10403C090E29093F104423041F0433050
:1059000051F0413069F49091F104946007C0909196
:10591000F104986003C09091F1049C609093F104AD
:1059200041E050E04217530718F4440F551FFACFD7
:105930009091F10440315105F1F050F4423051059D
:10594000B1F048305105E1F421E02093F00413C098
:105950004034510591F04038510539F0403251053D
:1059600079F421E02093F00408C0936007C091E02F
:105970009093F00405C0916001C092609093F1048F
:105980002CB59091F104922B9CBD9091F004992339
:1059900019F09DB591609DBD80931201E82FE295AD
:1059A000EF70F0E031A1282F2F7081E090E001C06E
:1059B000880F2A95EAF7932F982B91A392A18095AF
:1059C000892382A381E0089580E00895CF93DF9337
:1059D0008EBD0E94A322EC010DB407FC0AC00E94F8
:1059E000A3228C1B9D0B84369105B0F38EEF9FEFA5
:1059F00002C08EB590E0DF91CF910895CF93DF93F1
:105A00001EBC0E94A322EC010DB407FC0AC00E9438
:105A1000A3228C1B9D0B84369105B0F38EEF9FEF74
:105A200002C08EB590E0DF91CF9108950F931F9340
:105A3000CF93DF93EC018C01060F171FC017D1071E
:105A400031F089910E94E62C97FD03C0F7CF80E0EA
:105A500090E0DF91CF911F910F9108950F931F93C5
:105A6000CF93DF93EC018C01060F171FC017D107EE
:105A700031F00E94FE2C97FD04C08993F7CF80E09F
:105A800090E0DF91CF911F910F91089580911201C5
:105A90008F3F19F1E82FE295EF70F0E031A1282F48
:105AA0002F7081E090E001C0880F2A95EAF7932FCC
:105AB000982B91A392A1892B82A38FEF809312013F
:105AC0008DB58E7F8DBD9CB58091F1048095892325
:105AD0008CBD1092F1041092F004089597FB072EEC
:105AE00016F4009407D077FD09D00E94822D07FCA0
:105AF00005D03EF4909581959F4F089570956195DE
:105B00007F4F0895AA1BBB1B51E107C0AA1FBB1FF3
:105B1000A617B70710F0A61BB70B881F991F5A9539
:105B2000A9F780959095BC01CD010895EE0FFF1F58
:105B30000590F491E02D0994FC0188279927E894B9
:105B400021912032E9F3293010F02E30C8F32B32A6
:105B500041F02D3239F4689404C00E94FB2D820F6D
:105B6000911D219120532A30C0F31EF49095819508
:105B70009F4F0895FB01DC0102C005900D9241503A
:105B80005040D8F70895FB01DC018D9105908019F4
:105B90000110D9F3990B0895FB01DC0105900D92DA
:105BA0000020E1F70895FC0105900020E9F78095B9
:105BB00090958E0F9F1F0895FB01DC0102C001909C
:105BC0000D9241505040D8F70895FB01DC010D9033
:105BD0000020E9F7119701900D920020E1F7089558
:105BE000FC0181E090E00190061609F4CF0100204D
:105BF000D1F7019708957AE0979F902D879F802D88
:105C0000910D11240895AEE0B0E0E9E0FEE20C94BD
:105C100014310D891E898F89988D26E02C831A8373
:105C2000098397FF02C080E090E801979E838D83EF
:105C3000AE01455E5F4F698D7A8DCE0101960E945F
:105C4000332E4D815E8157FD0AC02F813885421762
:105C500053070CF49A01F801E20FF31F10822E96FD
:105C6000E4E00C943031ABE0B0E0E9E3FEE20C9408
:105C700006316C017B018A01FC0117821682838147
:105C800081FFCCC1CE0101963C01F6019381F70161
:105C900093FD859193FF81917F01882309F4BAC117
:105CA000853239F493FD859193FF81917F0185328F
:105CB00029F4B60190E00E942A30E7CF912C212CE4
:105CC000312CFFE1F315D8F08B3279F038F48032C3
:105CD00079F08332A1F4232D20611DC08D3261F053
:105CE000803369F4232D216016C0832D8260382E05
:105CF000E32DE4603E2E2AC0F32DF8601DC037FC72
:105D00002DC020ED280F2A3040F08E32B9F436FC39
:105D100081C1232D2064322E19C036FE06C08AE0D0
:105D2000989E200D1124922E11C0EAE02E9E200D87
:105D30001124222EF32DF0623F2E08C08C3621F460
:105D4000832D8068382E02C0883641F4F70193FD18
:105D5000859193FF81917F018111B3CF982F9F7D12
:105D60009554933028F40C5F1F4F9FE399830DC027
:105D7000833631F0833771F0833509F059C021C083
:105D8000F801808189830E5F1F4F88248394912CB2
:105D9000530113C02801F2E04F0E511CF801A080FE
:105DA000B18036FE03C0692D70E002C06FEF7FEF57
:105DB000C5010E941F304C018201F32DFF773F2E59
:105DC00016C0280122E0420E511CF801A080B180CB
:105DD00036FE03C0692D70E002C06FEF7FEFC50192
:105DE0000E9414304C01F32DF0683F2E820133FCE9
:105DF0001BC0822D90E088169906B0F4B60180E2AF
:105E000090E00E942A302A94F4CFF50137FC859166
:105E100037FE81915F01B60190E00E942A30211087
:105E20002A9421E0821A91088114910471F7E8C044
:105E3000843611F0893641F5F80137FE07C06081DC
:105E40007181828193810C5F1F4F08C060817181D5
:105E5000072E000C880B990B0E5F1F4FF32DFF765A
:105E60003F2E97FF09C090958095709561957F4F63
:105E70008F4F9F4FF0683F2E2AE030E0A3010E9431
:105E80006630882E861845C0853731F4232D2F7E45
:105E9000B22E2AE030E025C0932D997FB92E8F369F
:105EA000C1F018F4883579F0B5C0803719F088371B
:105EB00021F0B0C0E92FE061BE2EB4FE0DC0FB2D75
:105EC000F460BF2E09C034FE0AC0292F2660B22E0E
:105ED00006C028E030E005C020E130E002C020E14B
:105EE00032E0F801B7FE07C0608171818281938141
:105EF0000C5F1F4F06C06081718180E090E00E5FF3
:105F00001F4FA3010E946630882E8618FB2DFF7755
:105F10003F2E36FE0DC0232D2E7FA22E891458F45D
:105F200034FE0BC032FC09C0832D8E7EA82E05C026
:105F3000B82CA32C03C0B82C01C0B92CA4FE0FC0F0
:105F4000FE01E80DF11D8081803321F49A2D997EA8
:105F5000A92E09C0A2FE06C0B394B39404C08A2D32
:105F6000867809F0B394A3FC11C0A0FE06C0B21459
:105F700088F4280C922C9B180EC0B21460F4B60161
:105F800080E290E00E942A30B394F7CFB21418F464
:105F90002B1802C0982C212CA4FE10C0B60180E35F
:105FA00090E00E942A30A2FE17C0A1FC03C088E73F
:105FB00090E002C088E590E0B6010CC08A2D86789A
:105FC00059F0A1FE02C08BE201C080E2A7FC8DE285
:105FD000B60190E00E942A30891438F4B60180E3BB
:105FE00090E00E942A309A94F7CF8A94F301E80D4A
:105FF000F11D8081B60190E00E942A308110F5CF1A
:10600000222009F442CEB60180E290E00E942A30BC
:106010002A94F6CFF6018681978102C08FEF9FEF19
:106020002B96E2E10C942231FC0105906150704006
:106030000110D8F7809590958E0F9F1F0895FC0151
:106040006150704001900110D8F7809590958E0FA7
:106050009F1F08950F931F93CF93DF93FB0123811D
:1060600021FD03C08FEF9FEF2CC022FF16C0468199
:106070005781248135814217530744F4A081B181AF
:106080009D012F5F3F4F318320838C932681378181
:106090002F5F3F4F3783268314C08B01EC01FB0138
:1060A0000084F185E02D0995892BE1F6D80116963B
:1060B0008D919C911797019617969C938E931697A6
:1060C000CE01DF91CF911F910F910895FA01AA2778
:1060D000283051F1203181F1E8946F936E7F6E5F2B
:1060E0007F4F8F4F9F4FAF4FB1E03ED0B4E03CD0D9
:1060F000670F781F891F9A1FA11D680F791F8A1FBC
:10610000911DA11D6A0F711D811D911DA11D20D022
:1061100009F468943F912AE0269F11243019305DDC
:106120003193DEF6CF010895462F4770405D4193CD
:10613000B3E00FD0C9F7F6CF462F4F70405D4A331A
:1061400018F0495D31FD4052419302D0A9F7EACFE2
:10615000B4E0A6959795879577956795BA95C9F711
:1061600000976105710508959B01AC010A2E069404
:106170005795479537952795BA95C9F7620F731FBD
:10618000841F951FA01D0895F999FECF92BD81BD72
:10619000F89A992780B50895A8E1B0E042E050E070
:1061A0000C94F830262FF999FECF92BD81BDF89A54
:1061B000019700B4021639F01FBA20BD0FB6F8944B
:1061C000FA9AF99A0FBE08950396272F0E94D330AA
:1061D0000E94D230252F0E94D330242F0C94D3302C
:1061E0000196272F0E94D3300C94D230DC01CB01D2
:1061F000FC01F999FECF06C0F2BDE1BDF89A3196D7
:1062000000B40D9241505040B8F708952F923F923C
:106210004F925F926F927F928F929F92AF92BF92B6
:10622000CF92DF92EF92FF920F931F93CF93DF9362
:10623000CDB7DEB7CA1BDB0B0FB6F894DEBF0FBEBF
:10624000CDBF09942A88398848885F846E847D840C
:106250008C849B84AA84B984C884DF80EE80FD800E
:106260000C811B81AA81B981CE0FD11D0FB6F89484
:10627000DEBF0FBECDBFED0108955058BB27AA2742
:106280000E9455310C94C8320E94BA3238F00E94F4
:10629000C13220F039F49F3F19F426F40C94B73240
:1062A0000EF4E095E7FB0C94B132E92F0E94D9324D
:1062B00058F3BA17620773078407950720F079F43B
:1062C000A6F50C94FB320EF4E0950B2EBA2FA02D00
:1062D0000B01B90190010C01CA01A0011124FF2793
:1062E000591B99F0593F50F4503E68F11A16F0408E
:1062F000A22F232F342F4427585FF3CF469537958D
:106300002795A795F0405395C9F77EF41F16BA0B51
:10631000620B730B840BBAF09150A1F0FF0FBB1FFF
:10632000661F771F881FC2F70EC0BA0F621F731F48
:10633000841F48F4879577956795B795F7959E3FA5
:1063400008F0B0CF9395880F08F09927EE0F979536
:10635000879508950E948D3208F481E008950E9487
:10636000C3310C94C8320E94C13258F00E94BA3234
:1063700040F029F45F3F29F00C94B13251110C9494
:10638000FC320C94B7320E94D93268F39923B1F3EE
:10639000552391F3951B550BBB27AA27621773074B
:1063A000840738F09F5F5F4F220F331F441FAA1FDF
:1063B000A9F335D00E2E3AF0E0E832D0915050409B
:1063C000E695001CCAF72BD0FE2F29D0660F771F49
:1063D000881FBB1F261737074807AB07B0E809F02F
:1063E000BB0B802DBF01FF2793585F4F3AF09E3FB4
:1063F000510578F00C94B1320C94FC325F3FE4F319
:10640000983ED4F3869577956795B795F7959F5FF6
:10641000C9F7880F911D9695879597F90895E1E042
:10642000660F771F881FBB1F621773078407BA07A1
:1064300020F0621B730B840BBA0BEE1F88F7E095FC
:1064400008950E94E13288F09F5798F0B92F99275C
:10645000B751B0F0E1F0660F771F881F991F1AF04F
:10646000BA95C9F714C0B13091F00E94FB32B1E087
:1064700008950C94FB32672F782F8827B85F39F086
:10648000B93FCCF3869577956795B395D9F73EF4E8
:1064900090958095709561957F4F8F4F9F4F089590
:1064A000E89409C097FB3EF49095809570956195AE
:1064B0007F4F8F4F9F4F9923A9F0F92F96E9BB2764
:1064C0009395F695879577956795B795F111F8CFE0
:1064D000FAF4BB0F11F460FF1BC06F5F7F4F8F4F4B
:1064E0009F4F16C0882311F096E911C0772321F041
:1064F0009EE8872F762F05C0662371F096E8862FD9
:1065000070E060E02AF09A95660F771F881FDAF72F
:10651000880F9695879597F90895990F0008550F5C
:10652000AA0BE0E8FEEF16161706E807F907C0F019
:1065300012161306E407F50798F0621B730B840B21
:10654000950B39F40A2661F0232B242B252B21F4FB
:1065500008950A2609F4A140A6958FEF811D811D9B
:10656000089597F99F6780E870E060E008959FEFD5
:1065700080EC089500240A941616170618060906DA
:10658000089500240A9412161306140605060895A9
:10659000092E0394000C11F4882352F0BB0F40F431
:1065A000BF2B11F460FF04C06F5F7F4F8F4F9F4F71
:1065B000089557FD9058440F551F59F05F3F71F0F3
:1065C0004795880F97FB991F61F09F3F79F087955A
:1065D0000895121613061406551FF2CF4695F1DFE3
:1065E00008C0161617061806991FF1CF8695710573
:1065F000610508940895E894BB2766277727CB01A7
:1066000097F908950E948D3208F48FEF08950E9443
:106610001A330C94C8320E94BA3238F00E94C13248
:1066200020F0952311F00C94B1320C94B732112460
:106630000C94FC320E94D93270F3959FC1F3950FF0
:1066400050E0551F629FF001729FBB27F00DB11DF6
:10665000639FAA27F00DB11DAA1F649F6627B00D86
:10666000A11D661F829F2227B00DA11D621F739F6F
:10667000B00DA11D621F839FA00D611D221F749F7D
:106680003327A00D611D231F849F600D211D822FC4
:10669000762F6A2F11249F5750409AF0F1F08823EB
:1066A0004AF0EE0FFF1FBB1F661F771F881F915018
:1066B0005040A9F79E3F510580F00C94B1320C94E4
:1066C000FC325F3FE4F3983ED4F386957795679567
:1066D000B795F795E7959F5FC1F7FE2B880F911D42
:1066E0009695879597F90895FB01DC0104C08D917B
:1066F0000190801921F441505040C8F7881B990B34
:066700000895F894FFCF9C
:1067060001BC204F211C21F8200A21BB203075FF37
:106716000101FF0020406080A0C0E000F4F1F09687
:106726009091373697404732D903920360032B0482
:1067360044045D04818283E200E900EA00B500B604
:1067460000B700CD008301CC008A0192019401219B
:1067560002230224022502260227022A02B300B4DB
:10676600006F0070004C0052004D00300041542B69
:10677600424C45504F5745524C4556454C3D256475
:02678600000011
:00000001FF
